:0300000002375074
:0C37500078FFE4F6D8FD75814D02379734
:1013EF0020000A3C2E2E2E3E004950436F6E6E6534
:1013FF0063745245510A004950436F6E6E656374B2
:10140F00000A49504E6F41434B210A003E432C5670
:10141F002C52432CC0E4E0EFF2E5F020D1E8EDEAE6
:10142F00EEEC49500A003E432C4D41432C253032FF
:10143F0062583A25303262583A25303262583A258E
:10144F00303262583A25303262583A25303262587B
:10145F002C4D414320E0E4F0E5F10A003E432C56C9
:10146F0045522C20332E3220EEF220257320257387
:10147F002CC2E5F0F1E8FF20495020ECEEE4F3EB4D
:10148F00FF0A004A756C2033302032303132003180
:10149F00353A32373A3335003E432C4C442C5052B8
:1014AF004F473A20202020202020202020202020BD
:1014BF00202020202020202020202020202020201D
:1014CF00202020202020202020202020202020200D
:1014DF0020202020202020202020202020202020FD
:1014EF0020202020202020202CC4E0F2E020EFF04C
:1014FF00EEF8E8E2EAE828F4E0E9EB290A003E2AF0
:10150F002C312CCEF1EDEEE2EDFBE520EFE0F0E03B
:10151F00ECE5F2F0FB20F1E5F2E5E2EEE3EE20E898
:10152F00EDF2E5F0F4E5E9F1E00A003E412C41303F
:10153F00312C2562752E2562752E2562752E25623A
:10154F00752C495020E0E4F0E5F120E0E4E0EFF203
:10155F00E5F0E00A003E412C4130322C2562752E19
:10156F002562752E2562752E2562752C495020E057
:10157F00E4F0E5F120EEF1ED2E20F1E5F0E2E5F0FB
:10158F00E00A003E412C4130332C2562752E256236
:10159F00752E2562752E2562752C495020E0E4F0DA
:1015AF00E5F120F0E5E72E20F1E5F0E2E5F0E00AC5
:1015BF00003E412C4130342C2562752E2562752E4C
:1015CF002562752E2562752CCCE0F1EAE020F1E55D
:1015DF00F2E80A003E412C4130352C2562752E254C
:1015EF0062752E2562752E2562752CD8EBFEE70AE3
:1015FF00003E2A2C312CC4EEEF2E20EFE0F0E0EC71
:10160F00E5F2F0FB20F1E5F2E5E2EEE3EE20E8EDA6
:10161F00F2E5F0F4E5E9F1E00A003E422C533031F7
:10162F002C2562752CC6E4E0F2FC20E7E0EFF0EE2B
:10163F00F1E020F1EEE5E4E8EDE5EDE8FF20EEF274
:10164F0020F1E5F0E2E5F0E00A003E422C533032A3
:10165F002C2562752CCEE1ECE5ED20F120F1E5F0C3
:10166F00E2E5F0EEEC20E1E5E720EAE2E8F2E0ED7A
:10167F00F6E8E90A003E422C5330332C2562752CD4
:10168F00CFE5F0E5E7E0EFF3F1EA20EFF0E820EF48
:10169F00EEF2E5F0E520F1E2FFE7E820F120F1E5D9
:1016AF00F0E2E5F0EEEC0A003E422C5330382C25E8
:1016BF0062752CCCE5E4EBE5EDEDFBE9204950201C
:1016CF00EAE0EDE0EB28E7E0E4E5F0E6EAE020E42D
:1016DF00EE203520F1E5EA290A003E454E440A0086
:1016EF000A44756D70582020202020303020303172
:1016FF002030322030332030342030352030362027
:10170F0030372030382030392030412030422030DF
:10171F0043203044203045203046000A3A003A201A
:10172F00000A000A44756D704420202020203030BC
:10173F0020303120303220303320303420303520EB
:10174F0030362030372030382030392030412030AB
:10175F00422030432030442030452030460045722F
:10176F0072206B657900526420656570726F6D0A27
:10177F00005264204D454D0A00526420436F64654A
:10178F000A00577269746520436F64650A004465E7
:10179F006275674950204F4E0A004465627567496C
:1017AF0050204F46460A004465627567557365724F
:1017BF00204F6E0A00446562756755736572204F3E
:1017CF0046460A0044656275674D7367204F6E0A7F
:1017DF000044656275674D7367204F46460A0043A4
:1017EF006F6E666967206C6F636B210A00577220FA
:1017FF00656570726F6D0A002053617665206565AF
:10180F0070726F6D210A00457272204D41432100A5
:10181F004C6F61643E3E002A00CEF8E8E1EAE00A30
:10182F0000202D202575282575290A003C413031CF
:10183F003D003C4130323D003C4130333D003C41A6
:10184F0030343D003C4130353D003C21003C5330AD
:10185F00313D003C5330323D003C5330333D003C72
:10186F005330353D003C5330383D003C5330363D0E
:01187F000068
:063F64000114000112002F
:103FC200C28E438910E4F58B758DB8D2ABD28E22A6
:03001B000236C0EA
:1036C000C0E0C083C082C0D0C28E758B00758DB83B
:1036D000201E0675A61E75A6E10512D21AE5146015
:1036E0000205140517E517540F7051E513D3940123
:1036F00040021513D226E517543F7012D218906677
:103700008EE0600A04F0E0D394B44002D21E9066CA
:1037100087E0600204F0906104E0600214F09066BB
:103720008FE0D394014003E014F0301D020515E54D
:1037300016D394644004D21E80020516E511D3947A
:103740000140021511D28ED0D0D082D083D0E03289
:1008DB00C2237D027C007F07123F478F27E52764E9
:1008EB006060097D017F60123EDFD223E4FDFC7F57
:1008FB000B123F478F27E52730E6097D04E4FF12F3
:10090B003F03D2237D017C007F07123F478F27E5F2
:10091B00277008FD7FFF123EDFD2233023031260C6
:10092B0000C288C2A8C2AA75890012362490634AF5
:10093B007403F0A374CCF0E4906349F090668CF0F0
:10094B00A3F0122FCC123582C21E123C7CD223C2D2
:10095B0025C2249065777408F09062B57424F0E496
:10096B00A3F090633FE09062B7F0906340E0906239
:10097B00B8F0906341E09062B9F0906342E090620E
:10098B00BAF0906343E09062BBF0906344E09062F6
:10099B00BCF0751301E4906578F0C21FC220C22130
:1009AB00C222202318AF27FE7D031230B2E4FF12C0
:1009BB0034D27E137FEFE4FBFDFC1228FB90668E96
:1009CB00E060037401F0E4906104F0F51590657636
:1009DB00F0F516123FC275A70775A61E75A6E1D2D4
:1009EB00AFE4F516906104E07003122CFD90668F56
:1009FB00E06401701D9080007410F09080A874FF6B
:100A0B00F0A3F0A3F0A3F0E490668FF0D223C224FE
:100A1B00C225908008E0F52730E405D21F7410F052
:100A2B00E52730E508D2219080087420F0E52730C7
:100A3B00E608D2209080087440F0E515C39403407B
:100A4B0019908002E4F0908001F0908000F0E515A1
:100A5B0094064006E4F515123C7C9080A0E07003F0
:100A6B00123AF29080B8E07003123A789080D0E09E
:100A7B007003123C20908000E07013301F10122A7C
:100A8B0002906332EFF0D394004003120026908063
:100A9B0002E07006908000E06005D21D0209ECC2F6
:100AAB001DE4F515906104E060030209EC202312AC
:100ABB00906579E0600C7E137FF1122EE4E4906573
:100ACB0079F03021121224FB906332EFF0D39400B3
:100ADB004005E0FF12401B202003020C6B12237415
:100AEB00906332EFF070030209EC906376E054BF31
:100AFB00247F7003020BC6147003020B9E2402604A
:100B0B0003020C0D2023077E137FF8122EE42027FF
:100B1B0003020C6B90634EE0FF7006906352E06033
:100B2B0061906683E0FEB50722A3E0FF90634FE080
:100B3B00B50718906685E0FF906350E0B5070C9001
:100B4B006686E0FF906351E06F6037906352E06E12
:100B5B006003020C6B906684E0FF906353E06F6060
:100B6B0003020C6B906685E0FF906354E06F6003AB
:100B7B00020C6B906686E0FF906355E06F6003029A
:100B8B000C6BC21B9065787401F012401D7513013C
:100B9B00020C6B90668EE060037401F090667BE054
:100BAB00FF906378E06F6003020C6B90667BE00450
:100BBB00F0E4F513906576F0020C6B301B03020C1E
:100BCB006B906345E070030209EC9062B4E060083F
:100BDB00906356741EF080069063567403F01240B7
:100BEB001CD21BE4F513906576F090668704F0E455
:100BFB0090667AF0A3F02023677E147F06122EE412
:100C0B00805E90668EE060037401F0301B5290633F
:100C1B0076E020E74B906378E0FF90667AE0FE6F1A
:100C2B00600D906682E07007EE146F703380139046
:100C3B00667AE004F0906332E0FFD3940440031231
:100C4B002C029060007482F0A37401F0906378E042
:100C5B00906002F07E607F007D031238630209EC26
:100C6B00201B03020D8EE513706E1221DAEF602349
:100C7B007E647F76906477E02404FD12386390667F
:100C8B0082E07009906356E0F5130209ECE4F5136A
:100C9B000209EC906687E0D3943C403C906682E07E
:100CAB0070369062B4E0703090668704F0123416A0
:100CBB00E4906476F0A37412F090667BE090647815
:100CCB00F0A374FDF090610563A20190647A63A2B6
:100CDB00017F12121F288098123FAE8F27E527B491
:100CEB0001159060007483F0E4A3F07E607F007DBB
:100CFB00021238630209ECE527D39401401C906083
:100D0B00007483F0A37401F0E52724FEA3F07E604A
:100D1B007F007D031238630209ECE5136401600365
:100D2B000209EC906576E004F02023077E147F1017
:100D3B00122EE4906576E0FFD39401400B9063563E
:100D4B00E0941E5003E004F0EFC39405400DC21B6A
:100D5B00E4906578F012401D0209EC7C667D83906F
:100D6B00634AE0FAA3E0FB7F021239F47E647F76DC
:100D7B00906477E02404FD123863906356E0F5131A
:100D8B000209ECE513640160030209EC906578E05D
:100D9B0014604624FE6042147003020E812404602A
:100DAB00030209ECE4F5152027139065787404F021
:100DBB00906576E05401F07513010209EC90800206
:100DCB007410F0E4906578F090657604F07513126A
:100DDB0090668374FFF00209EC906683E070030267
:100DEB000E6B9064767480F09064787401F0E4A3D9
:100DFB00F0A304F0A37430F0A3747BF0E4F5277434
:100E0B007D2527F582E43464F583747DF0747E25AB
:100E1B0027F582E43464F583E4F0E5272407906436
:100E2B0077F07C667D8390634AE0FAA3E0FB7F0258
:100E3B001239F47E647F76E5272409FD123863901E
:100E4B006682E0601B12401CD21BE4F513906576A2
:100E5B00F090668704F0E490667AF0A3F00209EC58
:100E6B00302707E4906578F080069065787404F07D
:100E7B007513120209EC9080027410F07513039035
:100E8B006576E06401FFF09065787401F0EF7019FE
:100E9B00906352E06013FCA3E0FDA3E0FEA3E0FF30
:100EAB00906683121CF40209EC90634EE0FCA3E005
:100EBB00FDA3E0FEA3E0FF906683121CF40209EC95
:020ECB0080FEA7
:010ECD002202
:10002600906377E0B444047F0180027F009063769A
:10003600E0B447047E0180027E00EE5F604A906372
:100046003FE0906378F0906340E0906379F09063CE
:1000560041E090637AF0906342E090637BF09063B6
:1000660043E090637CF0906344E090637DF090639E
:10007600777452F09062AE63A2019080A863A201E9
:100086007F06121F280208D1906332E0C3940850FD
:10009600030208DA90633FE0FF906378E06F600345
:1000A6000208DA906340E0FF906379E06F60030234
:1000B60008DA906341E0FF90637AE06F600302081C
:1000C600DA906342E0FF90637BE06F60030208DA38
:1000D600906343E0FF90637CE06F60030208DA9070
:1000E6006344E0FF90637DE06F60030208DA90638B
:1000F60077E06444701A9080A8E0B4FF139062AE73
:1001060063A2019080A863A2017F06121F288010B7
:100116009062B2E09080ACF09062B3E09080ADF077
:1001260090668EE060037401F090668F7464F090C0
:1001360063777452F0906376E0646D600302027830
:100146007BFF7A14791B1218E27BFF7A14793590BB
:10015600633FE0F530A3E0F531A3E0F532A3E0F527
:1001660033A3E0F534A3E0F5351218E27530FF75D8
:1001760031147532927533FF75341475359E7BFFD5
:100186007A14796B1218E27BFF7A1479A71218E2B7
:100196007BFF7A15790D1218E27BFF7A15793A9072
:1001A6006345E0F530A3E0F531A3E0F532A3E0F5D1
:1001B600331218E27BFF7A15796490634EE0F530CE
:1001C600A3E0F531A3E0F532A3E0F5331218E27BA4
:1001D600FF7A157992906352E0F530A3E0F531A3EA
:1001E600E0F532A3E0F5331218E27BFF7A1579C009
:1001F60090633BE0F530A3E0F531A3E0F532A3E0F0
:10020600F5331218E27BFF7A1579E3906337E0F550
:1002160030A3E0F531A3E0F532A3E0F5331218E29E
:100226007BFF7A1679001218E27BFF7A167929A2EB
:1002360027E433F5301218E27BFF7A167959906677
:1002460082E0F5301218E27BFF7A16798490668E8A
:10025600E0F5301218E27BFF7A1679B79062B4E0C7
:10026600F5301218E212334A7BFF7A1679E9121832
:10027600E222906376E0644C70737E167FEFFBFD9E
:10028600FC1228FB90637EE0F528A3E0F529E4F54F
:100296002BE528906380F0A3E529F07E177F2A7C62
:1002A600637D807B021228FBE4F52A852982852856
:1002B60083E0FF7480252AF582E43463F583EFF04A
:1002C6000529E52970020528052AE52AB410DC7EF1
:1002D600177F2D7C637D807B101228FB052BE52B79
:1002E600C3941040AC7E177F30122EE422906376C2
:1002F600E0646C7060F52C7E177F32FBFDFC1228E3
:10030600FBE4F52BE4906380F0A3E52CF07E177FE9
:100316002A7C637D807B021228FBE4F52AA82CE662
:10032600FF7480252AF582E43463F583EFF0052C0B
:10033600052AE52AB410E67E177F2D7C637D807B37
:10034600101228FB052BE52BC3940840B77E177FB8
:1003560030122EE422906376E0644B7061F52A74C5
:1003660068252AF582E43463F583E06032746825F3
:100376002AF582E43463F583E0F460237468252A61
:10038600F582E43463F583E0FF747E252AF582E482
:100396003463F583E0B50710052AE52AB408C09052
:1003A60061047432F00208D19063767421F0302330
:1003B600030208D17E177F6D122EE40208D19063E6
:1003C60076E0B4521A2023077E177F75122EE4902A
:1003D60063767472F07E637F767D081237DC229036
:1003E6006376E0644970452023077E177F80122ECE
:1003F600E490637EE0F528A3E0F529E4F52A852953
:1004060082852883E0FF7480252AF582E43463F52B
:1004160083EFF00529E52970020528052AE52AB4A7
:1004260080DC7E637F767D8A1237DC22906376E0FD
:10043600644370462023077E177F88122EE490635C
:100446007EE0F528A3E0F529E4F52A8529828528AA
:1004560083E493FF7480252AF582E43463F583EF01
:10046600F00529E52970020528052AE52AB480DB6E
:100476007E637F767D8A1237DC22906376E0645A4B
:1004860070532023077E177F91122EE490637EE03F
:10049600F528A3E0F5297C637D807B80AF29AE2813
:1004A600123DD2E4F52A852982852883E493FF74D8
:1004B60080252AF582E43463F583EFF00529E529E2
:1004C60070020528052AE52AB480DB7E637F767DE7
:1004D6008A1237DC22906376E06444600302056C7E
:1004E60090637EE0FF644470030208D1EFB4310CE0
:1004F600C2237E177F9D122EE40208D190637EE010
:10050600B4300CD2237E177FA9122EE40208D190B4
:10051600637EE0B4320CD2247E177FB6122EE4023C
:1005260008D190637EE0B4330CC2247E177FC412D8
:100536002EE40208D190637EE0B4340CD2257E17F7
:100546007FD3122EE40208D190637EE0B4350CC24C
:10055600257E177FE0122EE40208D190637EE0FF2D
:1005660012401A0208D1906104E070132023077E1E
:10057600177FEE122EE49063767421F00208D19074
:1005860061047432F0906376E0FFB45104C2AF8028
:10059600FEEF645770452023077E177FFC122EE47A
:1005A60090637FE0906332F0E4F52A906332E0FFD7
:1005B600E52AC39F40030208D17480252AF582E408
:1005C6003463F583E0FF90637EE0252A24ADF5824F
:1005D600E43461F583EFF0052A80D0906376E06419
:1005E60053600302068E2023077E187F07122EE42F
:1005F60090633FE0FF9061B6E06F703C906340E02F
:10060600FF9061B7E06F7030906341E0FF9061B892
:10061600E0B50724906342E0FF9061B9E0B50718A2
:10062600906343E0FF9061BAE0B5070C906344E045
:10063600FF9061BBE06F60169063767421F0302303
:10064600030208D17E187F16122EE40208D1E4F5C3
:100656002AE4F51674AD252AF582E43461F583E0C3
:10066600FDAF2A123E65052AE52AC394FE40E2C282
:10067600AFE4907FF0F0A3F0907FFD74AAF0A3742E
:10068600FFF0A37455F080FE906376E0644F705AD5
:1006960090637EE0F528A3E0F529E5294528700A50
:1006A6002023077E187F1F122EE42023077E187F43
:1006B60026122EE4E4F52A7480252AF582E43463B2
:1006C600F583E0852982852883F00529E5297002CE
:1006D6000528052AE52AB480DE90668DE02480F0A0
:1006E60090668CE03400F00208D1906376E06445B1
:1006F600707490637EE0FEA3E0FF907FF0EEF0A3BF
:10070600EFF0D39400EE94044038907FF0E0FEA31F
:10071600E0FF90668CE0FCA3E0FD9FEC9E4023E4A6
:100726002FFFEE3401FED3ED9FEC9E5015C2AF9025
:100736007FFD74AAF0A374FFF0A37455F0E4F5A747
:1007460080FE7E187F28122EE47BFF7A187930907F
:100756007FF0E0F530A3E0F53190668CE0F532A34A
:10076600E0F5331218E2906376E0646560030208F0
:10077600DA90637EE0FFA3E0907FF0CFF0A3EFF086
:10078600E4F528F529D3907FF1E09529907FF0E0F4
:1007960095284021E4F5162529FFE5283478FE7BC7
:1007A60080AD29AC28123DD274802529F529E4357F
:1007B60028F52880D07E187F3B1238EAEF4E60205D
:1007C600120003906345EFF0120003906346EFF0CA
:1007D600120003906347EFF0120003906348EFF0B6
:1007E6007E187F411238EAEF4E60201200039063B4
:1007F6004EEFF012000390634FEFF0120003906388
:1008060050EFF0120003906351EFF07E187F47120D
:1008160038EAEF4E6020120003906352EFF01200A8
:1008260003906353EFF0120003906354EFF012004D
:1008360003906355EFF07E187F4D1238EAEF4E6055
:100846002012000390633BEFF012000390633CEF2D
:10085600F012000390633DEFF012000390633EEF49
:10086600F07E187F531238EAEF4E60201200039094
:100876006337EFF0120003906338EFF01200039035
:100886006339EFF012000390633AEFF0E4F52AE4DF
:10089600F516E52A04FF7437252AF582E43463F554
:1008A60083E0FD123E65052AE52AC3944340E0C273
:1008B600AFE4907FF0F0A3F0907FFD74AAF0A374EC
:1008C600FFF0A37455F0E4F5A780FE7E637F767D86
:0408D600081237DCF1
:0108DA0022FB
:103D9A00AE07EEC39430400BEED394395005EE24AF
:103DAA00D0FF22EEC39461400BEED394665005EE29
:103DBA0024A9FF22EEC39441400BEED3944650054A
:083DCA00EE24C9FF22AF06221E
:103F80009062ADE004F070069062ACE004F09062E4
:0A3F9000ACE0FEA3E0FF123D1F228B
:10000300123F80123D9AEFC454F0FEC006123F80A7
:08001300123D9AD0E02FFF22FC
:103BC300E4906AC8F0123F80906AC9EFF0C3943062
:103BD3004018E0FFD394395011906AC8E02405F5EA
:103BE30082E43461F583EFF08011906AC8E0240524
:103BF300F582E43461F583E4F0800C906AC8E00454
:103C0300F0E0D3940840BE752B00752C00752D0091
:0C3C1300E4F52E7B017A61790512203661
:013C1F002282
:0438EA008E2D8F2E62
:1038EE009062ACE4F0A374FFF0123F80EF606EF4D0
:1038FE00606B852E82852D83E493B507EC752F01C1
:10390E00E52E252FF582E4352DF583E49360259081
:10391E0062ADE0252FFF9062ACE03400FE123D1F39
:10392E00E52E252FF582E4352DF583E493B50704B6
:10393E00052F80CCE52E252FF582E4352DF583E479
:10394E009370A6E52F24FFFFE434FFFE9062ADE0F6
:10395E002FF09062ACE03EF07E007F0122E4FEFF8D
:01396E002236
:102FCC007E187F591238EAEF4E70037F01227E186B
:102FDC007F5C1238EAEF4E600C123F80EF24D02455
:102FEC00FF92278002D2277E187F621238EAEF4EBA
:102FFC00600C123F80EF24D0906682F08005E49044
:10300C006682F07E187F681238EAEF4E600C123F31
:10301C0080EF24D090668EF08005E490668EF07E72
:10302C00187F6E1238EAEF4E600C123F80EF24D0FE
:10303C0024FF92198002C2197E187F741238EAEFAD
:10304C004E600C123F80EF24D09062B4F08005E407
:10305C009062B4F090633F63A20190667C63A2011E
:10306C007F06121F2830193B7E187F7A1238EAEF40
:10307C004E603012000390667CEFF01200039066F5
:10308C007DEFF012000390667EEFF0120003906665
:10309C007FEFF0120003906680EFF0120003906651
:0630AC0081EFF07F00221D
:103CD600906577E0C3947C40027F0A906577E0FEAA
:103CE60004F074B52EF582E43462F583EFF0BF0A72
:103CF60027906577E0FF04F074B52FF582E434620F
:103D0600F583E4F0906577E0FF12396F906577747C
:093D160008F09062B6E004F0220E
:100ECE003E2A2C312CCFE0F0E0ECE5F2F0FB20E0F6
:100EDE00F1E8EDF5F0EEEDEDEEE3EE20EFEEF0F2F3
:100EEE00E02E20D0E5E6E8EC20F0E0E1EEF2FB208B
:100EFE002D20EFE0EAE5F2EDFBE920EFEE20554480
:100F0E005020E820EAE2E0E7E8EFEEF2EEEAEEE269
:100F1E00FBE920EFEE205443500A003E432C4B30A9
:100F2E00362C25732CD2E5EAF3F9E8E920F0E5E654
:100F3E00E8EC0A003E4C2C4930312C256C752CD136
:100F4E00EAEEF0EEF1F2FC20EEE1ECE5EDE02C3510
:100F5E00302C3130302C3330302C3630302C313286
:100F6E0030302C323430302C343830302C3936305E
:100F7E00302C31393230302C33383430302C353748
:100F8E003630302C3131353230300A003E422C4969
:100F9E0030322C2562752CD3EFF0E0E2EBE5EDE874
:100FAE00E520EFEEF2EEEAEEEC20EFF0E820EFE5D2
:100FBE00F0E5E4E0F7E520285254532D435453292D
:100FCE000A003E532C4930332C2562752CC7E0E4C1
:100FDE00E5F0E6EAE020F1F2E0F0F2E020EFE5F0F5
:100FEE00E5E4E0F7E8282A3130ECF1290A003E4228
:100FFE002C4930342C2562752CD0E5E6E8EC20EF38
:10100E00E5F0E5E4E0F7E8203720E1E8F20A003EFB
:10101E00422C4930352C2562752CCFE5F0E5E4E005
:10102E00F7E020F120EAEEEDF2F0EEEBFCEDFBEC5A
:10103E0020E1E8F2EEEC0A003E422C4930362C2537
:10104E0062752CCAEEEDF2F0EEEBFCEDFBE920E161
:10105E00E8F2202D20F7E5F2EDEEF1F2FC0A003E6B
:10106E00422C415030372C2562752CC6E4E0F2FC40
:10107E0020EAE2E8F2E0EDF6E8FE20EEF220F3F1EF
:10108E00F2F0EEE9F1F2E2E00A003E422C4150307D
:10109E00382C2562752CCAE2E8F2E8F0EEE2E0F2B6
:1010AE00FC20EFE0EAE5F2FB20EEF220F3F1F2F0A5
:1010BE00EEE9F1F2E2E00A003C21003C4930313D1C
:1010CE00003C4930323D003C4930333D003C493014
:1010DE00343D003C4930353D003C4930363D003C06
:1010EE00415030373D003C415030383D000A536589
:1010FE006E64204B56543A20202020000ACFF0E593
:10110E00E2FBF8E5EDE8E520ECE0EAF12E20E4EB79
:10111E00E8EDFB20EFE0EAE5F2E020EDE020EEF274
:10112E00EFF0E0E2EAF321000ACFE5F0E5EFEEEBB7
:10113E00EDE5EDE8E520E1F3F4E5F0E020EDE0206B
:10114E00EEF2EFF0E0E2EAF321000A546F4164643C
:10115E003A20202020202020000A53656E64205063
:10116E0061636B65743A20000A43524320657272C4
:10117E006F7221202020000ACEF2E2E5F7E0FE2079
:10118E00EDE020E7E0E3F0F3E7EAF321000A526531
:10119E0063204B5654000A526563206F6B2120204A
:1011AE002020202000496E69745443500A004C6977
:1011BE007374656E5443500A00534F434B5F544350
:1011CE00505F45535441424C49534845440A000A26
:1011DE002D3E20000A3C2D20005443500055445013
:1011EE000000112332465765748C9DAFBECADBE9F1
:1011FE00F810013322564775649C8DBFAEDACBF9D9
:10120E00E82130021367764455ADBC8E9FEBFAC8C9
:10121E00D93120120377665445BDAC9E8FFBEAD8B8
:10122E00C94253617004152736CEDFEDFC8899ABA9
:10123E00BA5243716014053726DECFFDEC9889BB98
:10124E00AA6372405125340617EFFECCDDA9B88A89
:10125E009B7362504135241607FFEEDCCDB9A89A78
:10126E008B8495A7B6C2D3E1F008192B3A4E5F6D69
:10127E007C9485B7A6D2C3F1E018093B2A5E4F7D58
:10128E006CA5B48697E3F2C0D129380A1B6F7E4C49
:10129E005DB5A49687F3E2D0C139281A0B7F6E5C38
:1012AE004DC6D7E5F48091A3B24A5B69780C1D2F29
:1012BE003ED6C7F5E49081B3A25A4B79681C0D3F18
:1012CE002EE7F6C4D5A1B082936B7A48592D3C0E09
:1012DE001FF7E6D4C5B1A092837B6A58493D2C1EF8
:1012EE000F0089129B24AD36BF48C15AD36CE57EE0
:1012FE00F78108931AA52CB73EC940DB52ED64FF67
:10130E0076028B109926AF34BD4AC358D16EE77C56
:10131E00F5830A9118A72EB53CCB42D950EF66FD46
:10132E0074048D169F20A932BB4CC55ED768E17A36
:10133E00F3850C971EA128B33ACD44DF56E960FB26
:10134E0072068F149D22AB30B94EC75CD56AE37816
:10135E00F1870E951CA32AB138CF46DD54EB62F906
:10136E007008811A932CA53EB740C952DB64ED7606
:10137E00FF89009B12AD24BF36C148D35AE56CF7E6
:10138E007E0A8318912EA73CB542CB50D966EF74D6
:10139E00FD8B029910AF26BD34C34AD158E76EF5C6
:1013AE007C0C851E9728A13AB344CD56DF60E972B6
:1013BE00FB8D049F16A920BB32C54CD75EE168F3A6
:1013CE007A0E871C952AA338B146CF54DD62EB7096
:1013DE00F98F069D14AB22B930C74ED55CE36AF186
:0113EE007886
:103F6A0052669000000000000000000000000000FF
:053F7A00000000000042
:103EB80074B42549F582E43467F583EFF005499039
:103EC80067AFE549F064646005E549B4E408D208E1
:073ED8006349805349802279
:01401A002283
:030023000227CBE6
:0B27CB00C0E0C083C082C0D075D018F1
:1027D60020980302287F751401AE99200218EE6432
:1027E60002600302287D301005AF1E123EB8754602
:1027F60005D20202287D300F1EC20F301007AF1E11
:10280600123EB8806FAF49054974B42FF582E4349F
:1028160067F583EEF0805DBE090C301005AF1E1221
:102826003EB8D20F804EBE020D534980301045AFE0
:102836001E123EB8803EEE6403701F301007AF1EB6
:10284600123EB880069067AFE549F0634980534968
:1028560080C202D208754600801A301007AF1E12D9
:102866003EB88010AF49054974B42FF582E4346749
:10287600F583EEF0754605C29830996E30036930DF
:102886001107309704D200805F9066A4E0FFE54A06
:10289600C39F400FC203D214200B02D216C20BD222
:1028A600968045AF4A054A74B42FF582E43468F53C
:1028B60083E0F54B300919534B7F30012820D008AF
:1028C600200422634B80801D30041A634B808015E0
:1028D600300112E54B524B300406A2D0929B800584
:0C28E600A2D0B3929B854B99C299D2AF4F
:0928F200D0D0D082D083D0E032B6
:10334A007BFF7A0E79CE1218E23010147530FF75B1
:10335A0031117532E77BFF7A0F79291218E2801250
:10336A007530FF7531117532EB7BFF7A0F792912AF
:10337A0018E29069B4E0FEA3E0FFC3E49FFFE49E75
:10338A00FEAB07FA3395E0F9F87F007E8C7D0A7C64
:10339A0000121C438F338E328D318C307BFF7A0FB3
:1033AA0079421218E27BFF7A0F799AA211E433F577
:1033BA00301218E27BFF7A0F79D08547301218E273
:1033CA007BFF7A0F79FCA209E433F5301218E27B0D
:1033DA00FF7A10791DA201E433F5301218E27BFF5F
:1033EA007A107946A204E433F5301218E27BFF7AA8
:1033FA0010796DA212E433F5301218E27BFF7A10CD
:0C340A007998A20AE433F5301218E2228F
:102B06007E107FC61238EAEF4E70037F01227E10D8
:102B16007FC91238EAEF4E6023123BC3A804A90509
:102B2600AA06AB077F007E8C7D0A7C00121C43122E
:102B36001CD59069B4EEF0A3EFF0800A9069B474E6
:102B4600FFF0A374B8F07E107FCF1238EAEF4E6024
:102B56000C123F80EF24D024FF92118002C2117E16
:102B6600107FD51238EAEF4E6007123BC38F4780BD
:102B760003E4F5477E107FDB1238EAEF4E600C1255
:102B86003F80EF24D024FF92098002C2097E107F85
:102B9600E11238EAEF4E600C123F80EF24D024FF9A
:102BA60092018002C2017E107FE71238EAEF4E6082
:102BB6000C123F80EF24D024FF92048002C2047ED0
:102BC600107FED1238EAEF4E600E123F80EF24D0F0
:102BD60024FF920592128004C205C2127E107FF471
:102BE6001238EAEF4E600E123F80EF24D024FF9297
:0C2BF60005920A8004C205C20A7F00227A
:10358200C203C216C208C202C20FE4F54A9066A480
:10359200F0F549F514C200D297D2969067B0F0C206
:1035A20006C2159066A27409F0A3F0C209C204C251
:1035B20001C213C211E4F547F546D2149069B474FE
:1035C200FFF0A374B8F0C20AC205C212122B069011
:1035D20067A57401F0C2ADE4F5C9D2CDD2CCC2C99F
:1035E200C2CAF5CDF5CC9069B4E0F5CBA3E0F5CA3B
:1035F20085CBCD85CACCE4F59830010C200909535E
:1036020087BFD29FD29E8002D29E438740C29FC272
:10361200ACC298C29975B81075B710D2CAD29CD2F2
:02362200AC22D8
:103F9A00E54D6FFF9012EF93654CF54DEF9011EFE1
:033FAA0093F54C40
:013FAD0022F1
:01401B002282
:04266C008E2A8F2BF8
:10267000E4F52CF54DF54CAA06A9077B018B308AB1
:10268000318932121BF5042532F532E43531F5314A
:1026900030050F9067A6E0AB30AA31A932121BF5C6
:1026A000800D9066A3E0AB30AA31A932121BF575FC
:1026B0003001852A31852B320D0DE4FEEEC39D508D
:1026C00018AB300532E532AA317002053114F91227
:1026D0001BDCFF123F9A0E80E3AB300532E532AAD5
:1026E000317002053114F9E54D121BF5AB30AA31FA
:1026F000A932E54C121BF50D0D300E0F9067B1E0BD
:10270000A3E0FAA3E08A2EF52F8006752E68752FB8
:10271000B4753001852A31852B32852F82852E8331
:102720007402F0052FE52F7002052E052CE4FEEE55
:10273000C39D504EAB30AA31A932121BDCF52D647B
:1027400002600BE52D64036005E52DB40913852FA8
:1027500082852E837409F0052FE52F7002052E0562
:102760002C852F82852E83E52DF0052FE52F700215
:10277000052E052C74012532F532E43531F5310E84
:1027800080AD852F82852E837403F0052FE52F7091
:1027900002052E052C906696E0FCA3E0FDA3E0FE6A
:1027A000A3E0FFE4FAF9F8EF2401FFEA3EFEE93D79
:1027B000FDE83CFC906696121CF49067B17401F041
:0A27C000A3E52EF0A3E52FF0AF2CE7
:0127CA0022EC
:10341600E4FF9066A3E0FE7D000FED2405F582E44F
:103426003461F583EEF00F74052401F582E434610E
:10343600F583E4F07C667D95FEED1DAA0470011C03
:10344600F5828A83E0FBAA070F74052AF582E43425
:1034560061F583EBF00EBE04E07C667D99E4FEED3B
:103466001DAA0470011CF5828A83E0FBAA070F746B
:10347600052AF582E43461F583EBF00EBE04E07CA8
:10348600667D9DE4FEED1DAA0470011CF5828A830B
:10349600E0FBAA070F74052AF582E43461F583EB95
:1034A600F00EBE04E07C667DA1E4FEED1DAA04706C
:1034B600011CF5828A83E0FBAA070F74052AF582B0
:0B34C600E43461F583EBF00EBE04E07F
:0134D10022D8
:05001E00C299D29922F5
:01401C002281
:103D6100AD072010337E677FA512266C9066A4EF05
:103D7100F0D203E4F54A30250D7E107FFB7C687D8F
:103D8100B4E0FB1228FBC296301103D20022E547B2
:093D91006003F5112212001E224C
:022C02008F2819
:102C0400301003022CFCE528D394FA40122025034B
:102C1400022CFC7E117F0AE4FBFDFC1228FB22300F
:102C240003427A6979B37B01C003C002C001906793
:102C3400B1E0A3E0FAA3E07E002528F9EE3AFAC356
:102C4400D082D083D0E0E99582EA95834012202592
:102C540003022CFC7E117F36E41BFDFC1228FB22B0
:102C6400C2ACD20E906379E09066A3F0300E177E6A
:102C7400637F78E52824FCFD12266C8F299066A4D6
:102C8400E02529F080117E637F78E52824FCFD127D
:102C9400266C9066A4EFF0A21282055005754805D3
:102CA400D215D203200E17E4F54AC296301104D28D
:102CB40000800BE5476004F511800312001E3025E7
:102CC40031300E1E7E117F589067B1E0A3E0FAA365
:102CD400E0AC02C39529FDEC9400FCAB291228FB5F
:102CE40080107E117F677C687DB49066A4E0FB123F
:082CF40028FBC20EC216D2AC8F
:012CFC0022B5
:1021DA00200603300B037F00222008030223693004
:1021EA0010037F0022C208E4906476F09067AFE0A3
:1021FA00FF547F24FCF528906477F090667BE0908A
:10220A006478F0EF5480FF24B5F582E43467F583EF
:10221A00E0906479F074B42FF582E43467AD82FCFF
:10222A00E4F54DF54CFE9067AFE0547FF9EEC399A3
:10223A0050140DEDAA0470010C14F5828A83E0FF94
:10224A00123F9A0E80E0E54C454D60443025197ED8
:10225A00117F769067AFE0548024B4F582E4346746
:10226A00AD82FCAB011228FB90669AE0FCA3E0FD6C
:10227A00A3E0FEA3E0FFE4FAF9F8EF2401FFEA3E47
:10228A00FEE93DFDE83CFC90669A121CF4022369C3
:10229A003005249067AFE05480FF24B4F582E4341B
:1022AA0067F583E09067A5F074B52FF582E434678B
:1022BA00F583E09067A6F0E5287039C215F54890D5
:1022CA0067A6E0B4E01E7490F0200503022369D2E9
:1022DA00062025030223697E117F85E4FBFDFC129B
:1022EA0028FB807B3025787E117F9BE4FBFDFC1266
:1022FA0028FB806B9067AFE0548024B6F582E43403
:10230A0067F58363A20190647A63A201AF28121F62
:10231A002830251C7E117FA49067AFE0FB548024EF
:10232A00B4F582E43467AD82FCEB547FFB1228FBE0
:10233A00906692E0FCA3E0FDA3E0FEA3E0FFE4FACE
:10234A00F9F8EF2401FFEA3EFEE93DFDE83CFC9086
:10235A006692121CF4A20A82055002D206D21730E3
:09236A001705C2177F01227F0054
:012373002247
:103E060030082DC2083010289067AFE0FF54802498
:103E1600B4F582E43467F58363A2019069BA63A2BC
:103E260001EF547FFF121F289067AFE0547FFF22F7
:033E36007F0022E8
:01401D002280
:102CFD003018469080E8E0700F123B603025077E5B
:102D0D00117FB3122EE4C2109080E8E0B40E129041
:102D1D0080037408F03025077E117FBC122EE4C2AB
:102D2D00109080E8E0B4060F20100C3025077E11BE
:102D3D007FC7122EE4D210C21830105C2003071288
:102D4D0031938F288003E4F528E528602F30250C7A
:102D5D007E117FDD7C697DBAFB1228FB9069BA6319
:102D6D00A2019068B463A201AF28121F289066A437
:102D7D00E528F0E4F54AD203C296D299123E068FA9
:102D8D0028E5286013122DF430250D7E117FE27C8D
:102D9D00697DBAAB281228FB300008209705C200C8
:102DAD0012001EE511B40106E4F51112001E3026C5
:102DBD0023C226E546600BD54608634980534980FA
:102DCD00C20230120FE548600BD54808E4F54AD22F
:102DDD0003754805A20A8206500C200309E4FF1270
:062DED003D61C206D20B9D
:012DF30022BD
:103FAE003010037F0022301608201505C2167F013F
:043FBE00227F00223C
:103C7C009080007480F090633763A201F583F58225
:103C8C0063A2017F08121F2890633F63A2019080FA
:103C9C008863A2017F0A121F289080927407F0A3F8
:103CAC0074D0F0A37406F0906349E0FF9080B1F0FB
:103CBC009080E1EFF09080957455F0A3F090800027
:0A3CCC007401F090800974F0F022FA
:103AF200908009E04410F09080A0E070609080A176
:103B02007482F09080A874FFF0A3F0A3F0A3F07F7A
:103B1200039080AEEFF0A374CBF09080007402F0BB
:103B2200906ABA121D0000000000906ABAE090800C
:103B320040F0906ABBE0908041F0906ABCE09080D7
:103B420042F0906ABDE0908043F0A3E4F0A3F0A3BA
:0D3B5200F0A3F0908018F0A3F0A3F0A3F012
:013B5F002243
:103C2000908009E04440F09080D17482F07F03904E
:103C300080DEEFF0A374CCF09080027402F0906A02
:103C4000BE121D0000000000906ABEE0908058F097
:103C5000906ABFE0908059F0906AC0E090805AF07E
:103C6000906AC1E090805BF0A3E4F0A3F0A3F0A31E
:0B3C7000F0908030F0A3F0A3F0A3F070
:013C7B002226
:103A7800908009E04420F09080B8E0706C9080B9A4
:103A88007482F07F039080C6EFF07FCDA3EFF07FC4
:103A9800039080C4EFF0A374CDF09080C074FFF061
:103AA800A3F0A3F0A3F09080017402F0906AC21210
:103AB8001D0000000000906AC2E090804CF0906AFF
:103AC800C3E090804DF0906AC4E090804EF0906A18
:103AD800C5E090804FF0A3E4F0A3F0A3F0A3F0902A
:093AE8008024F0A3F0A3F0A3F088
:013AF10022B2
:1039F4008C288D29A907EAFDE975F018A424ACFFE9
:103A0400E5F034808F82F583EDF0EBFDE975F01875
:103A1400A4FFAEF024ACFBEE34808B82F583A3EDDF
:103A2400F08529828C83E0FDEF24A8FFEE3480FE2C
:103A34008F82F583EDF08529828C83A3E08F828EBB
:103A440083A3F0852982852883A3A3E0FDE975F08B
:103A540018A424A8FFE5F03480FE8F82F583A3A385
:103A6400EDF08529828C83A3A3A3E08F828E83A3A8
:043A7400A3A3F022F6
:0637DC008D2DAB07AA06CB
:1037E200908000E030E5079065797401F022906ADC
:1037F200BAE0FCA3E0FDA3E0FEA3E0F5318E308D3C
:103802002F8C2EAE02AF038E838F8263A201E5302E
:10381200540744C0F58385318263A201AF2D121F84
:103822009AE4FCFDFEE531252DF531EE3530F5301B
:10383200ED352FF52FEC352EF52E908040E52EF04C
:10384200A3E52FF0A3E530F0A3E531F090800074FA
:1038520020F0AF31AE30AD2FAC2E906ABA121CF40C
:013862002243
:063863008D28AB07AA0648
:10386900908002E030E5079065797403F022906A50
:10387900BEE0FCA3E0FDA3E0FEA3E0F52C8E2B8DBA
:103889002A8C29AE02AF038E838F8263A201E52BB6
:10389900540744D0F583852C8263A201AF28121FF7
:1038A9009AE4FCFDFEE52C2528F52CEE352BF52BAD
:1038B900ED352AF52AEC3529F529908058E529F0C6
:1038C900A3E52AF0A3E52BF0A3E52CF09080027480
:1038D90020F0AF2CAE2BAD2AAC29906ABE121CF495
:0138E90022BC
:0234D2008F2841
:1034D400908001E030E5099065797402F07F002264
:1034E400906AC2E0FCA3E0FDA3E0FEA3E0F52C8E0D
:1034F4002B8D2A8C2990667C63A201E52B5407440A
:10350400C8F583852C8263A2017F06121FB0E52CC7
:103514002406F52CE4352BF52BE4352AF52AE4357D
:1035240029F52990657A63A201E52B540744C8F56F
:1035340083852C8263A201AF28121FB0E4FCFDFE38
:10354400E52C2528F52CEE352BF52BED352AF52A1F
:10355400EC3529F52990804CE529F0A3E52AF0A360
:10356400E52BF0A3E52CF09080017420F0AF2CAE95
:0D3574002BAD2AAC29906AC2121CF4AF28BE
:013581002227
:102A02009081E0E0F52805280528052805280528F5
:102A120005280528052805280528908010E0F52BB3
:102A2200A3E0F52CA3E0F52DA3E0F52E9081E1E0E3
:102A3200F52805280528052805280528052805283C
:102A4200052805280528908014E0F52FA3E0F5302D
:102A5200A3E0F531A3E0F532E531B52D08E532B555
:102A62002E037F0022E4F528E531540744E0F58384
:102A720085328263A20190637663A2017F08121FEE
:102A8200E090637863A2019062AE63A2017F0612B6
:102A92001F28906376E0F529A3E0F52AE4F5289053
:102AA2006376E0702AA3E024F8F528E53154074460
:102AB200E0F58385328274082582F582E43583F558
:102AC2008363A20190637663A201AF28121FE0AE76
:102AD20029E4FCFDE532252AF532E5313EF531EDFA
:102AE2003530F530EC352FF52F908014E52FF0A31B
:102AF200E530F0A3E531F0A3E532F09080007440B8
:032B0200F0AF2809
:012B050022AD
:102374009081E6E0F5280528052805280528052884
:1023840005280528052805280528908028E0F52B30
:10239400A3E0F52CA3E0F52DA3E0F52E9081E7E072
:1023A400F5280528052805280528052805280528D1
:1023B40005280528052890802CE0F52FA3E0F530AA
:1023C400A3E0F531A3E0F532E4F528E531B52D0AB3
:1023D400E532B52E05C2200224E0E531540744F06D
:1023E400F58385328263A20190637663A2017F083C
:1023F400121FE0906376E0F529A3E0F52AE52A456B
:102404002970099080027410F07F0022906683E0A6
:10241400FFF46030906378E06F60030224A7906655
:1024240084E0FF906379E06F7079906685E0FF90B7
:10243400637AE06F706D906686E0FF90637BE06F77
:102444006031805F906378E0906683F0906379E018
:10245400906684F090637AE0906685F090637BE008
:10246400906686F090637CE0FFA3E090634ACFF02F
:10247400A3EFF0906376E0702AA3E024F8F528E552
:1024840031540744F0F58385328274082582F5823D
:10249400E43583F58363A20190637663A201AF28D8
:1024A400121FE0AE29E4FCFDE532252AF532E531C0
:1024B4003EF531ED3530F530EC352FF52FAF2EAE3E
:1024C4002DAD2CAC2BAB32AA31A930A82FD3121CC2
:1024D400E340099080027410F07F002290802CE584
:1024E4002FF0A3E530F0A3E531F0A3E532F09080BE
:0624F400027440F0AF2865
:0124FA0022BF
:1024FB009081E3E0F52805280528052805280528FF
:10250B000528052805280528052890801CE0F52BB3
:10251B00A3E0F52CA3E0F52DA3E0F52E9081E4E0EC
:10252B00F528052805280528052805280528052848
:10253B00052805280528908020E0F52FA3E0F5302D
:10254B00A3E0F531A3E0F532E4F528E531B52D0A2A
:10255B00E532B52E05C221022651E531540744E878
:10256B00F58385328263A20190600463A2017F0E22
:10257B00121FF6906004E0F529A3E0F52A90600C99
:10258B00E0FFF4604A90667CE0FEEF6E7079A3E0AA
:10259B00FF90600DE06F706F90667EE0FF90600EB5
:1025AB00E06F706390667FE0FF90600FE06F705795
:1025BB00906680E0FF906010E06F704B906681E05A
:1025CB00FF906011E06F703FE4906013F080089013
:1025DB00601374FFF0D2D9906004E0702AA3E0245A
:1025EB00F2F528E531540744E8F583853282740E01
:1025FB002582F582E43583F58363A2019060046341
:10260B00A201AF28121FF6AE29E4FCFDE532252A04
:10261B00F532E5313EF531ED3530F530EC352FF552
:10262B002FAF2EAE2DAD2CAC2BAB32AA31A930A8CF
:10263B002FD3121CE35006E52A452970099080011F
:10264B007410F07F0022908020E52FF0A3E530F08E
:10265B00A3E531F0A3E532F09080017440F0AF2890
:01266B00224C
:042EE4008E2D8F2E72
:102EE800908000E030E5079065797401F022906ADF
:102EF800BAE0FCA3E0FDA3E0FEA3E0F5348E338D39
:102F0800328C31E534FFE5335407FEE42FF530EE1B
:102F180034C0F52F853082F5837423F00530E53011
:102F28007002052F532FC7F582852F83740AF00589
:102F380030E5307002052F532FC790633F63A2011D
:102F4800852F8385308263A2017F06121F9A74063B
:102F58002530F530E4352FF52F852D83852E8263B6
:102F6800A201852F8385308263A201121F7EE4FCB3
:102F7800FDFE906ABAE0F8A3E0F9A3E0FAA3E02F17
:102F8800FFEE3AFEED39FDEC38FCEF2408FFE43E95
:102F9800FEE43DFDE43CFC906ABA121CF4906ABA67
:102FA800E0908040F0906ABBE0908041F0906ABC6D
:102FB800E0908042F0906ABDE0908043F0908000FD
:032FC8007420F082
:012FCB0022E3
:0A28FB008E2D8F2E8C2F8D308B3127
:10290500908000E030E5079065797401F022906AC7
:10291500BAE0FCA3E0FDA3E0FEA3E0F5378E368D1B
:10292500358C34E537FFE5365407FEE42FF533EEF5
:1029350034C0F532853382F5837423F00533E533EE
:10294500700205325332C7F582853283740AF00569
:1029550033E533700205325332C790633F63A201FA
:1029650085328385338263A2017F06121F9A74061E
:102975002533F533E43532F532852D83852E826393
:10298500A20185328385338263A201121F7E8F38AF
:10299500EF2533F533E43532F532E5316017852F10
:1029A5008385308263A20185328385338263A201E8
:1029B500AF31121F9AE53824082531F531FFE4FCC3
:1029C500FDFEE5372FF537EE3536F536ED3535F5C0
:1029D50035EC3534F534908040E534F0A3E535F039
:1029E500A3E536F0A3E537F09080007420F0AF370B
:0C29F500AE36AD35AC34906ABA121CF45A
:012A010022B2
:06326F008E088F098D0A94
:10327500908000E030E5079065797401F022906A4E
:10328500BAE0FCA3E0FDA3E0FEA3E0F5108E0F8DF0
:103295000E8C0DE510FFE50F5407FEE42FF50CEE3F
:1032A50034C0F50B850C82F5837423F0050CE50C11
:1032B5007002050B530BC7F582850B83EBF0050CEC
:1032C500E50C7002050B530BC790633F63A20185A4
:1032D5000B83850C8263A2017F06121F9A74062553
:1032E5000CF50CE4350BF50B85088385098263A283
:1032F50001850B83850C8263A201AF0A121F9A74A4
:1033050008250AF50AFFE4FCFDFEE5102FF510EE91
:10331500350FF50FED350EF50EEC350DF50D9080ED
:1033250040E50DF0A3E50EF0A3E50FF0A3E510F0E1
:103335009080007420F0AF10AE0FAD0EAC0D906A0A
:04334500BA121CF4A8
:013349002261
:02396F008F4186
:10397100908000E030E5079065797401F022906A4B
:10398100BAE0FCA3E0FDA3E0FEA3E0F5458E448D83
:10399100438C42E545FFE5445407FEE42FFFEE3436
:1039A100C09062B563A201F5838F8263A201AF412A
:1039B100121F9AE4FCFDFEE5452541F545EE35442F
:1039C100F544ED3543F543EC3542F542908040E551
:1039D10042F0A3E543F0A3E544F0A3E545F0908070
:1039E100007420F0AF45AE44AD43AC42906ABA12C8
:0239F1001CF4C4
:0139F30022B1
:0630B2008E288F29AB05FA
:1030B800908000E030E5079065797401F022906A0D
:1030C800BAE0FCA3E0FDA3E0FEA3E0F52F8E2E8D71
:1030D8002D8C2CE52FFFE52E5407FEE42FF52BEE63
:1030E80034C0F52A852B82F5837423F0052BE52B54
:1030F8007002052A532AC7F582852A83EBF0052B2F
:10310800E52B7002052A90633F63A201852A838517
:103118002B8263A2017F06121F9A7406252BF52BBA
:10312800E4352AF52A532AC7E528852B82852A8380
:10313800F0052BE52B7002052A532AC7F582852A4C
:1031480083E529F0052BE52B7002052A532AC7E5EC
:103158002F240AF52FE4352EF52EE4352DF52DE430
:10316800352CF52C908040E52CF0A3E52DF0A3E557
:103178002EF0A3E52FF09080007420F0AF2FAE2E34
:0A318800AD2DAC2C906ABA121CF4B5
:01319200221A
:103B6000908009E04480F09080E97441F07F0990F2
:103B700080F6EFF0A37464F09080037402F09080FC
:103B800003E020E1F99069B6121D000000000090EA
:103B900069B6E0908064F09069B7E0908065F0903D
:103BA00069B8E0908066F09069B9E0908067F0A312
:103BB000E4F0A3F0A3F0A3F090803CF0A3F0A3F016
:023BC000A3F070
:013BC20022E0
:103193009081E9E0F529052905290529052905294E
:1031A30005290529052905290529908034E0F52AF3
:1031B300A3E0F52BA3E0F52CA3E0F52D9081EAE045
:1031C300F52905290529052905290529052905299C
:1031D300052905290529908038E0F52EA3E0F52F70
:1031E300A3E0F530A3E0F531E530B52C08E531B5C2
:1031F3002D037F0022AF31AE30AD2FAC2EAB2DAA05
:103203002CA92BA82AD3121CE3400AAF31AE2DEE12
:103213009FF529800AAF31EFF404AE2D2EF529E591
:1032230030540744E0F58385318263A2019069BA83
:1032330063A201AF2912200EE4FCFDFEE53125292E
:10324300F531EE3530F530ED352FF52FEC352EF524
:103253002E908038E52EF0A3E52FF0A3E530F0A300
:0B326300E531F09080037440F0AF29CB
:01326E00223D
:022DF4008F2925
:102DF6009080E8E0640660037FFF229069B6E0FCFD
:102E0600A3E0FDA3E0FEA3E0F52D8E2C8D2B8C2AEE
:102E1600E4FFFEFDFCAB2DAA2CA92BA82AC3121C8D
:102E2600E370609081F9E0F52A9069B6E0FCA3E0D2
:102E3600FDA3E0FEA3E0FFE4FAF9F8EF2401FFEAC0
:102E46003EFEE93DFDE83CFC9069B6121CF4906933
:102E5600B6E0FCA3E0FDA3E0FEA3E0FFE4F8EF2468
:102E660001FFEA3EFEE93DFDE83CFC9069B6121C16
:102E7600F4908064E0F52AA3E0F52BA3E0F52CA3FB
:102E8600E0F52D9069BA63A201E52C540744D8F504
:102E960083852D8263A201AF29121FC8E4FCFDFEC3
:102EA600E52D2529F52DEE352CF52CED352BF52BBD
:102EB600EC352AF52A908064E52AF0A3E52BF0A3E9
:102EC600E52CF0A3E52DF09080037420F0AF2DAE35
:0D2ED6002CAD2BAC2A9069B6121CF47F00C5
:012EE30022CC
:0A400800E4FEEEC39F50030E80F8A3
:01401200228B
:10362400E4F528E5282401FFE433FE123D1F743736
:103634002528F582E43463F583EFF00528E528C3F3
:10364400943F40DFE4F528E528247FFFE433FE12AD
:103654003D1F742D2528F582E43461F583EFF07461
:103664002D2528F582E43461F583E0FF6003B4FF7F
:103674001D742D2528F582E43461F5837420F074DB
:103684002E2528F582E43461F583E4F080090528C9
:10369400E528C3948040B0E49061ACF0F528AF28ED
:1036A4007E00123D1F74AD2528F582E43461F58354
:0B36B400EFF00528E528C394FE40E37A
:0136BF0022E8
:103F2700E4FDFCC3ED9FEC9E5015E4FBFA0BBB00D0
:0F3F3700010ABA01F8BB90F50DBD00010C80E442
:013F46002258
:0D3FE1004390014390025390FE5390FD2247
:0D3FEE005390FD5390FE439002439001223A
:0E3FD2005390FD439002E5905408FF5390FD7C
:013FE00022BE
:0D3FFB005390FD4390014390025390FD222E
:07401300AE071FEE70FA2258
:023E3900AD07D3
:103E3B00E4FC5390FDEDA804088002C333D8FC309A
:103E4B00E70543900180035390FE7F051240134317
:093E5B0090020CBC08DC5390FD40
:013E6400223B
:103E8F00E4FF5390FD7E07439002E59030E00D7400
:103E9F0001A806088002C333D8FC42075390FD1EC9
:083EAF00C3EE6480948050DF33
:013EB70022E8
:103E6500AB05AA07123FE17FA0123E39123FD2AF40
:103E750002123E39123FD2AF03123E39123FD2121F
:0A3E85003FEE7F0A7E00123F272265
:043D1F00AB07AA063E
:103D2300C3EB94FFEA9400400DE42BF58274773AD9
:103D3300F583E493FF22123FE17FA0123E39123F45
:103D4300D2AF03123E39123FD2123FE17FA1123E9E
:0D3D530039123FD2123E8F123FFB123FEE9D
:013D60002240
:023DD2008B2D37
:103DD400A2AF9228C2AF85A22E53A2FE8E838F82F9
:103DE40005A28C838D827409122024E52D53A2FE32
:103DF40043A22012202653A2DF852EA2A22892AF2E
:013E0400FFBE
:013E0500229A
:103F4700A2AF9228C2AF8C838D82EF12202443A2A6
:0C3F57002012202653A2DFA22892AFFF08
:013F6300223B
:023EDF008F282A
:103EE100A2AF9228C2AFE4F5838D8274061220241A
:103EF100E52843A22012202653A2DFA22892AF7FF9
:013F010001BE
:013F0200229C
:023F03008F2805
:103F0500A2AF9228C2AFE4F5838D82740A122024F1
:103F1500E52843A22012202653A2DFA22892AF7FD4
:013F2500019A
:013F26002278
:101E4D00A907E7FFA805EF93C3966008403B74FC14
:101E5D002FFF80F00F08EF93C3966008402B74FBA3
:101E6D002FFF80E00F08EF93C3966008401B74FAB4
:101E7D002FFF80D00F08EF93D3966008400B74F9B5
:101E8D002FFF80C01F1F1F1F1FEF54FEF80303F706
:101E9D00E893FC08E893FD08E893FE08E893FF2219
:101EAD0009E993C39D6008402974FB29F980F10964
:101EBD00E993C39E6008401A74FA29F980E209E992
:101ECD0093D39F6008400B74F929F980D319191920
:101EDD001919E9C313C313FF22740093F8ECC398C7
:101EED004024701F740193F8EDC398401970147459
:0E1EFD000293F8EEC398400E7009740393F838
:101F0B00EFC39840037F00227F0122EDF8E6F00833
:101F1B00A3DFFA22EDF8E0F608A3DFFA22E0A363D1
:101F2B00A201F0A363A201DFF475A2002263A20158
:101F3B00F0A363A20122E0A363A201F0A363A201B9
:101F4B00E0A363A201F0A363A201E463A201F0A3E7
:101F5B0063A201DFE175A20022E0A363A2016DFE83
:101F6B00936CFDEE058393FC158363A201DFEA7589
:101F7B00A200227F00E493A363A201F00F600CA3E5
:101F8B00E583C2E3F58363A20180EA75A20022E038
:101F9B00A363A201F0A3E583C2E3F58363A201DF90
:101FAB00EE75A20022E0A363A201F0A3E583C2E4D5
:101FBB00D2E3F58363A201DFEC75A20022E0A363F9
:101FCB00A201F0A3E58344F8C2E5F58363A201DF28
:101FDB00EC75A20022E583C2E3F583E0A363A201C3
:101FEB00F0A363A201DFEE75A20022E583C2E4D267
:0A1FFB00E3F583E0A363A201F0A365
:1020050063A201DFEC75A20022E58344F8F583E0C5
:10201500A363A201F0A363A201DFEE75A20022F97A
:1020250022C002C004C00612FFF0D006D004D002C0
:012035002288
:10375C000208DBE493A3F8E493A34003F68001F2A0
:10376C0008DFF48029E493A3F85407240CC8C3336E
:10377C00C4540F4420C8834004F456800146F6DF3D
:10378C00E4800B0102040810204080903F64E47E2A
:10379C00019360BCA3FF543F30E509541FFEE49332
:1037AC00A360010ECF54C025E060A840B8E493A3F9
:1037BC00FAE493A3F8E493A3C8C582C8CAC583CA24
:1037CC00F0A3C8C582C8CAC583CADFE9DEE780BEDC
:013F7F000041
:101BDC00BB010689828A83E0225002E722BBFE0207
:091BEC00E32289828A83E493223A
:101BF500BB010689828A83F0225002F722BBFE01CF
:021C0500F322C8
:101C070075F008758200EF2FFFEE33FECD33CDCC94
:101C170033CCC58233C5829BED9AEC99E582984017
:101C27000CF582EE9BFEED9AFDEC99FC0FD5F0D6F4
:101C3700E4CEFBE4CDFAE4CCF9A88222B800C1B91E
:101C47000059BA002DEC8BF084CFCECDFCE5F0CB5C
:101C5700F97818EF2FFFEE33FEED33FDEC33FCEB95
:101C670033FB10D703994004EB99FB0FD8E5E4F950
:101C7700FA227818EF2FFFEE33FEED33FDEC33FC3D
:101C8700C933C910D7059BE99A4007EC9BFCE99A31
:101C9700F90FD8E0E4C9FAE4CCFB2275F010EF2F76
:101CA700FFEE33FEED33FDCC33CCC833C810D70776
:101CB7009BEC9AE899400AED9BFDEC9AFCE899F8B1
:0E1CC7000FD5F0DAE4CDFBE4CCFAE4C8F92244
:0E1CD500C3E49FFFE49EFEE49DFDE49CFC2220
:101CE300EB9FF5F0EA9E42F0E99D42F0E89C45F057
:011CF30022CE
:0C1CF400ECF0A3EDF0A3EEF0A3EFF02263
:101D0000A8828583F0D083D082121D17121D17126E
:101D10001D17121D17E473E493A3C583C5F0C58393
:101D2000C8C582C8F0A3C583C5F0C583C8C582C82D
:011D30002290
:10188000E53C2430F8E6053C22782D302F027830F4
:10189000E475F001121DAD021BDC2028EB7F2ED277
:1018A000288018EF540F2490D43440D4FF302C0BF0
:1018B000EF24BFB41A0050032461FFE53D60021518
:1018C0003D0540E5407002053F302F0D782DE47551
:1018D000F001121DADEF021BF5023CD67403D22FAE
:1018E0008003E4C22FF53C8B2D8A2E892FE4F53D31
:1018F000F53FF540E53D60077F201218BB80F57588
:101900003EFFC229C228C22AC22BC22DC22EC2301B
:10191000121889FF700D302F057F001218CCAF40D0
:10192000AE3F22B4255FC2D5C22C121889FF24D045
:10193000B40A00501A75F00A783D30D50508B6FF94
:101940000106C6A426F620D5047002D22B80D92425
:10195000CFB41A00EF5004C2E5D22C021ACCD2291F
:1019600080C6D22880C0D22A80BCD2D580BAD22DDF
:1019700080B47F201218BB202A077401B53D0040B7
:10198000F1121880FF1218BB0218F4D230D22E8048
:1019900095121880FB121880FA121880F94A4B70C1
:1019A00006799D7A1B7BFF202A2EE53D602A7E006A
:1019B0008E82758300121D3160060EEE653E70F05A
:1019C000C2D5EBC0E0EAC0E0E9C0E0EE121B13D0E4
:1019D000E0F9D0E0FAD0E0FB121BDCFF60AAEBC01C
:1019E000E0EAC0E0E9C0E01218BBD0E02401F9D081
:1019F000E03400FAD0E0FBE53E0460DCD53ED9805F
:101A0000877BFF7A1B790FD22A809C79108002791C
:101A100008C22EC2308008D2D5790A8004790AC261
:101A2000D5E53E047002F53EE4FAFDFEFF12188093
:101A3000FC7B08202913121880FD7B1030280A1225
:101A40001880FE121880FF7B20EC3382D592D5508F
:101A500013C3E43028069FFFE49EFEE42029039D83
:101A6000FDE49CFCE4CBF8C229EC700CCFCECDCCCD
:101A7000E824F8F870F38017C3EF33FFEE33FEED80
:101A800033FDEC33FCEB33FB994002FB0FD8E9EB61
:101A9000302905F8D0E0C448B229C0E00AEC4D4E28
:101AA0004F78207B0070C2EAB53E0040BCC0E01217
:101AB0001B15D0F0D0E0202904C4C0E0C4B229C076
:101AC000F01218A4D0F0D5F0EB0218F4121E0C1985
:101AD00091531A0B5819624C195E421A0F4F1A177C
:0F1AE000441A17491977431A1D551A01461A015E
:101AEF00451A01471BBD5019662D196A2E198D2BEA
:101AFF00196E23198B201BA62A1926480000198559
:101B0F003F3F3F00790AA2D5202B14302D09B91081
:101B1F00020404B9080104A2D5202E0250010420AA
:101B2F002A68922AB53D005034C0E07F20302B192F
:101B3F007F30A22A722E722D500F121B6CC22AC236
:101B4F002EC22DC2307F30800F302D03E9C0E0123E
:101B5F0018BB302D03D0E0F9D0E0B53DCC302D17B8
:101B6F007F30B9100C1218BB7F58302C077F78804C
:101B7F0003B908031218BB302A057F2D0218BB7F4B
:101B8F00202030F87F2B202EF322922A80CF286E30
:101B9F00756C6C2900D2291218803029F8C2297867
:101BAF003D30D50108F60219262D50434958121819
:101BBF00802403B405004001E4901BB8931218ACC5
:0D1BCF00743A1218ACD22B753D04021A0BAB
:102036008B288A29892AE4F534F533F532F531F50A
:102046002FF530E52C452D452B6012EBC0E0EAC09C
:10205600E0E9C0E0AB2BAA2CA92D121DBDAB2805CB
:102066002AE52AAA297002052914F9121BDCF5357E
:10207600C394094007E535D3940D40E1E535642066
:1020860060DBE535B42D054330038016E535B42B0A
:1020960005433001800C74FF252AF52A74FF352983
:1020A600F529E52E60046410703FAB28AA29A92AF9
:1020B600121BDC64306009E52E702E752E0A80290D
:1020C600900001121D31FF64786004EFB458134389
:1020D6003001752E107402252AF52AE43529F529D2
:1020E6008007E52E7003752E08AB28052AE52AAA77
:1020F600297002052914F9121BDCF535C3946140D9
:102106000AE535D3947A50035335DF74D02535F577
:1021160035C3940A400CE5359411406D74F92535A4
:10212600F535E535D3952E50604330018534398534
:102136003338853237853136AF2E7E00E4FCFDAB71
:1021460034AA33A932A831121D5EC8ECC8C9EDC93C
:10215600CAEECACBEFCBE4FCFDFEEB2535F534EE3B
:102166003AF533ED39F532EC38F531AF34AE33ADFF
:1021760032FCAB39AA38A937A836D3121CE3500370
:102186000220EF4330040220EFE53020E003E48034
:102196002DE52C452D452B601EAB28E52A24FFF99D
:1021A600E52934FFFAEBC0E0EAC0E0E9C0E0AB2B7A
:1021B600AA2CA92D121DBDE53030E20774FFFFFEE3
:1021C600FDFC22E530AF34AE33AD32AC3130E10345
:0421D600021CD522F0
:101D3100BB010CE58229F582E5833AF583E0225067
:101D410006E92582F8E622BBFE06E92582F8E222B1
:0D1D5100E58229F582E5833AF583E49322CB
:101D5E00E88FF0A4CC8BF0A42CFCE98EF0A42CFC24
:101D6E008AF0EDA42CFCEA8EF0A4CDA8F08BF0A4A2
:101D7E002DCC3825F0FDE98FF0A42CCD35F0FCEB01
:101D8E008EF0A4FEA9F0EB8FF0A4CFC5F02ECD39C6
:0F1D9E00FEE43CFCEAA42DCE35F0FDE43CFC2233
:101DAD00FAE6FB0808E6F925F0F618E6CA3AF62237
:101DBD00BB011A89828A83D0F0D0E0F8D0E0F9D047
:101DCD00E0FAD0E0FBE8C0E0C0F0021E3B5016E99F
:101DDD00F8D083D082D0E0F9D0E0FAD0E0FBC08219
:101DED00C083021E32BBFE16E9F8D083D082D0E04C
:0F1DFD00F9D0E0FAD0E0FBC082C083021E44227E
:101E0C00D083D082F8E4937012740193700DA3A365
:101E1C0093F8740193F5828883E473740293686079
:061E2C00EFA3A3A380DF79
:091E3200EBF608EAF608E9F622D5
:091E3B00EBF0A3EAF0A3E9F022A8
:091E4400EBF208EAF208E9F222CF
:00000001FF
